:100000000C9462000C948A000C948A000C948A0070
:100010000C948A000C948A000C948A000C948A0038
:100020000C948A000C9446030C948A000C948A0069
:100030000C948A000C948A000C948A000C948A0018
:100040000C943B060C948A000C94C1070C948A0013
:100050000C948A000C948A000C948A000C948A00F8
:100060000C948A000C948A000000000024002700F1
:100070002A0000000000250028002B0000000000DE
:1000800023002600290004040404040404040202DA
:100090000202020203030303030301020408102007
:1000A0004080010204081020010204081020000012
:1000B0000007000201000003040600000000000029
:1000C0000000460911241FBECFEFD4E0DEBFCDBF34
:1000D00011E0A0E0B1E0ECE2F6E102C005900D9283
:1000E000AE38B107D9F713E0AEE8B1E001C01D9218
:1000F000AA3BB107E1F710E0C4ECD0E004C02297BE
:10010000FE010E94100BC23CD107C9F70E943F03B9
:100110000C94140B0C940000AF92BF92CF92DF921C
:10012000EF92FF920F931F93082FC62E67EAA62E19
:1001300063E0B62EC50140E050E060E070E020E0F2
:1001400030E00E94760ADD2410E054E0000F111F19
:100150005A95E1F7C02AD12AEE24D7FCE094FE2C70
:10016000C501B701A60120E030E00E94760A1F9188
:100170000F91FF90EF90DF90CF90BF90AF900895D8
:10018000AF92BF92CF92DF92EF92FF920F931F93A5
:10019000082FC62EE7EAAE2EE3E0BE2EC50140E1F1
:1001A00050E060E070E020E030E00E94760ADD245C
:1001B00010E074E0000F111F7A95E1F7C02AD12AF0
:1001C000EE24D7FCE094FE2CC501B701A60120E087
:1001D00030E00E94760A1F910F91FF90EF90DF9020
:1001E000CF90BF90AF90089585E061E00E94250711
:1001F00085E060E00E94250780E090E05F9A5F98CC
:10020000019620E180309207C9F7089585E061E00A
:100210000E94250784E060E00E942507E2E1F3E008
:1002200022813381C901807F9F7044E09595879535
:100230004A95E1F78EBD0DB407FEFDCF8EB5408126
:100240005181CA0180709F70892F990F990BA4E08A
:10025000220F331FAA95E1F7822B8EBD0DB407FE46
:10026000FDCF8EB54EBD0DB407FEFDCF8EB53497D4
:1002700082E0E239F807A1F684E061E00E942507F8
:1002800084E060E00E94250785E060E00E94250789
:10029000089585E061E00E94250784E060E00E9407
:1002A0002507E2E9F2E022813381C901807F9F7056
:1002B00074E0959587957A95E1F78EBD0DB407FEAC
:1002C000FDCF8EB540815181CA0180709F70892F0A
:1002D000990F990B54E0220F331F5A95E1F7822BA7
:1002E0008EBD0DB407FEFDCF8EB54EBD0DB407FE1D
:1002F000FDCF8EB5349782E0E231F807A1F684E0B5
:1003000061E00E94250784E060E00E94250785E007
:1003100060E00E942507089585E061E00E942507BE
:1003200084E060E00E942507E2E1F2E0228133816F
:10033000C901807F9F7044E0959587954A95E1F7C4
:100340008EBD0DB407FEFDCF8EB540815181CA012F
:1003500080709F70892F990F990BA4E0220F331F93
:10036000AA95E1F7822B8EBD0DB407FEFDCF8EB5A9
:100370004EBD0DB407FEFDCF8EB5349781E0E23956
:10038000F807A1F684E061E00E94250784E060E0C0
:100390000E94250785E060E00E942507089588B146
:1003A000836288B90E948C0145980E94F40088B14C
:1003B000836288B90E94490141980E94F40088B183
:1003C000836288B90E94060140980E94F400089553
:1003D000AF92BF92CF92DF92EF92FF920F931F9353
:1003E000CF93DF93FCE4AF2EF1E0BF2EEE24FF2489
:1003F000EFEFCE2EEFE0DE2E36C0D801ED918D016D
:10040000CE2FD0E0CC0FDD1FFE01EA56FE4FD18289
:10041000C0820E94CF010E94CF010E94CF01FE0145
:10042000EA56FD4FD182C0820E94CF010E94CF01C7
:100430000E94CF01CA5EDD4FD982C8820E94CF01DF
:100440000E94CF010E94CF010A151B05B1F6089446
:10045000E11CF11C68E0A62EB12CA00EB11EB8E084
:10046000EB16F10449F0870153E0000F111F5A9574
:10047000E1F70C5B1E4FC1CFDF91CF911F910F9120
:10048000FF90EF90DF90CF90BF90AF900895AF9224
:10049000BF92DF92EF92FF920F931F93DF93CF9360
:1004A00000D0CDB7DEB783E060E00E94250780E191
:1004B00061E00E942507EE24FF24DE2C83E061E04A
:1004C0000E94250788E060E00E94250788E061E03F
:1004D0000E942507AAE3AA2EA1E0BA2EAE0CBF1CEB
:1004E00017E08AE060E00E942507F5010081202FD7
:1004F00030E03A83298389E00E947207E981FA811A
:10050000E817F90781F089E00E947207F5018083FE
:10051000882329F4812F6D2D0E948C0004C0812F27
:100520006D2D0E94C0008AE061E00E94250728EF3F
:100530003FEFA20EB31E1150A0F683E060E00E94D0
:10054000250780E160E00E9425070894E11CF11C6A
:1005500038E0E316F10409F0B0CF0F900F90CF917F
:10056000DF911F910F91FF90EF90DF90BF90AF90C0
:1005700008950E94CF010E944702089588B18362C6
:1005800088B987B1836287B982E061E00E9405077C
:100590008BE061E00E9405078DE061E00E940507A5
:1005A00084E061E00E94050785E061E00E940507A4
:1005B00086E061E00E94050787E061E00E94050790
:1005C0008CE060E00E9405078AE061E00E94050778
:1005D0008AE061E00E9425078BE060E00E94250729
:1005E0008DE060E00E94250784E060E00E9425071E
:1005F00082E060E00E94250785E061E00E94250717
:1006000087E061E00E94250786E060E00E94250700
:1006100080E58CBD8DB58EB56AE070E080E090E03D
:100620000E94830689E060E00E9405078AE061E09D
:100630000E94050788E061E00E94050780E161E013
:100640000E94050783E061E00E94050787EA93E0C6
:1006500040E052EC61E070E00E94FE071092B000B2
:1006600083E08093B10081E0809370006AE070E0E5
:1006700080E090E00E9483060E94E80108950E94B5
:10068000AD060E94BE020E94B902FDCF1F920F92DA
:100690000FB60F921124BF92CF92DF92EF92FF928A
:1006A0000F931F932F933F934F935F936F937F937A
:1006B0008F939F93AF93BF93CF93DF93EF93FF936A
:1006C0007894BB24B39487EA93E00E94F7088823C8
:1006D00009F4B0C280914201882341F087EA93E097
:1006E0000E940B0980931903109242018091190313
:1006F000E82FF0E0CF0174E0959587957A95E1F7C2
:100700008530910509F439C1863091059CF4823019
:10071000910509F451C08330910524F4019709F043
:1007200089C21BC08330910509F488C0049709F081
:1007300081C2BAC08930910509F4F9C18A309105A6
:1007400024F4089709F076C283C18C30910509F42E
:1007500028C20D9709F06EC266C287EA93E00E9434
:10076000F708833008F466C287EA93E00E940B0919
:1007700064E0880F991F6A95E1F790938F01809349
:100780008E0187EA93E00E940B0954E0880F991FBD
:100790005A95E1F7909301018093000187EA93E075
:1007A0000E940B0944E0880F991F4A95E1F7909346
:1007B0009101809390013CC287EA93E00E94F70880
:1007C000882309F437C287EA93E00E940B09E82FD7
:1007D0008093180390E034E0959587953A95E1F77A
:1007E00080931603EF70E0931703F0E023E0EE0F21
:1007F000FF1F2A95E1F7E80FF91FEC5BFE4FE08140
:10080000F0E0EE0FFF1FDF01AA56BE4F80918E0170
:1008100090918F018D939C93DF01AA5EBD4F8091D3
:100820000001909101018D939C93EA56FD4F8091B8
:1008300090019091910191838083FAC187EA93E0BE
:100840000E94F708882309F4F5C187EA93E00E9423
:100850000B09E82F8093180390E014E09595879595
:100860001A95E1F780931603EF70E0931703F0E019
:10087000B3E0EE0FFF1FBA95E1F7E80FF91FEC5B4D
:10088000FE4FE081F0E0EE0FFF1FDF01AA56BE4FE2
:100890001D921C92DF01AA5EBD4F1D921C92EA566A
:1008A000FD4F11821082C4C187EA93E00E94F708CD
:1008B000882309F4BFC1809119038F7080931603B8
:1008C00087EA93E00E940B09809318039091160326
:1008D000292F30E0E0908E01F0908F01009100010F
:1008E00010910101C0919001D091910140E0682FD9
:1008F00070E0E3E0220F331FEA95E1F739C0E42FFF
:10090000F0E0CB01042E02C0959587950A94E2F79A
:1009100080FF17C0E20FF31FEC5BFE4FE081F0E0B9
:10092000EE0FFF1FDF01AA56BE4FED92FC92DF01D2
:10093000AA5EBD4F0D931C93EA56FD4FD183C08331
:1009400016C0E20FF31FEC5BFE4FE081F0E0EE0F0C
:10095000FF1FDF01AA56BE4F1D921C92DF01AA5E47
:10096000BD4F1D921C92EA56FD4F118210824F5FBF
:10097000483028F2409317035BC187EA93E00E9456
:10098000F708882309F456C1809119038F7080936A
:10099000170387EA93E00E940B0980931803909154
:1009A0001703692F70E0C0908E01D0908F01E09006
:1009B0000001F0900101009190011091910140E03F
:1009C000C82FD0E03FC0842F90E09E01042E02C0CB
:1009D000359527950A94E2F7FC0183E0EE0FFF1F9F
:1009E0008A95E1F720FF17C0E60FF71FEC5BFE4F7B
:1009F000E081F0E0EE0FFF1FDF01AA56BE4FCD925F
:100A0000DC92DF01AA5EBD4FED92FC92EA56FD4FEB
:100A10001183008316C0E60FF71FEC5BFE4FE081E9
:100A2000F0E0EE0FFF1FDF01AA56BE4F1D921C9291
:100A3000DF01AA5EBD4F1D921C92EA56FD4F118246
:100A400010824F5F483008F4BECF40931603F0C0C9
:100A500087EA93E00E94F708883008F4EBC0109210
:100A600016035FC087EA93E00E940B098093180386
:100A700050911603252F30E0E0908E01F0908F0109
:100A80000091000110910101C0919001D09191015C
:100A900040E0682F70E0E3E0220F331FEA95E1F7B2
:100AA00039C0E42FF0E0CB01042E02C09595879564
:100AB0000A94E2F780FF17C0E20FF31FEC5BFE4FD2
:100AC000E081F0E0EE0FFF1FDF01AA56BE4FED926E
:100AD000FC92DF01AA5EBD4F0D931C93EA56FD4FB9
:100AE000D183C08316C0E20FF31FEC5BFE4FE081A1
:100AF000F0E0EE0FFF1FDF01AA56BE4F1D921C92C1
:100B0000DF01AA5EBD4F1D921C92EA56FD4F118275
:100B100010824F5F483028F2409317035F5F509375
:100B2000160380911603883008F49CCF81C0E0FF43
:100B300022C060918E0170918F014091000150910F
:100B40000101209190013091910180E090E0FC0141
:100B5000EA56FE4F71836083FC01EA5EFD4F5183CC
:100B60004083FC01EA56FD4F318320830296803892
:100B7000910569F75DC080E090E0FC01EA56FE4F08
:100B800011821082FC01EA5EFD4F11821082FC018D
:100B9000EA56FD4F1182108202968038910569F75E
:100BA00047C0CF018F709070009721F0019709F036
:100BB0003FC018C0B092920183E00E94E70695956D
:100BC0008795959587958093940187EA93E040EE09
:100BD00050E060E070E020E030E00E94760A409152
:100BE000940117C0B092930184E00E94E7069595A6
:100BF0008795959587958093950187EA93E041EED7
:100C000050E060E070E020E030E00E94760A409121
:100C1000950150E060E070E087EA93E020E030E08A
:100C20000E94760A05C0EF70F070EE56FE4F1082FB
:100C3000B092420187EA93E00E94F708853608F0F7
:100C400042CDFF91EF91DF91CF91BF91AF919F91F5
:100C50008F917F916F915F914F913F912F911F9154
:100C60000F91FF90EF90DF90CF90BF900F900FBE4D
:100C70000F901F9018951F920F920FB60F9211248C
:100C80002F933F938F939F93AF93BF9380911E03B6
:100C900090911F03A0912003B09121033091220372
:100CA0000196A11DB11D232F2D5F2D3720F02D574B
:100CB0000196A11DB11D2093220380931E039093E2
:100CC0001F03A0932003B093210380911A039091F6
:100CD0001B03A0911C03B0911D030196A11DB11D22
:100CE00080931A0390931B03A0931C03B0931D03DE
:100CF000BF91AF919F918F913F912F910F900FBE18
:100D00000F901F901895EF92FF920F931F937B0106
:100D10008C018FB7F89440911E0350911F0360918E
:100D20002003709121038FBF2FB7F89480911E0389
:100D300090911F03A0912003B09121032FBF841B2A
:100D4000950BA60BB70BE816F9060A071B0760F709
:100D50001F910F91FF90EF900895789484B5826071
:100D600084BD84B5816084BD85B5826085BD85B54F
:100D7000816085BDEEE6F0E0808181608083E1E8FE
:100D8000F0E0808182608083808181608083E0E800
:100D9000F0E0808181608083E1EBF0E0808184601D
:100DA0008083E0EBF0E0808181608083EAE7F0E01F
:100DB0008081846080838081826080838081816083
:100DC00080838081806880831092C10008958F7035
:100DD000909143019295990F990F907C982B909345
:100DE0007C0080917A00806480937A0080917A0000
:100DF00086FDFCCF2091780040917900942F80E00F
:100E000030E0282B392BC9010895282F30E0C90183
:100E100086569F4FFC0194912A573F4FF9018491C8
:100E2000882391F0E82FF0E0EE0FFF1FE859FF4F05
:100E3000A591B491662329F48C91909589238C9384
:100E400008958C91892B8C930895482F50E0CA0106
:100E500082559F4FFC012491CA0186569F4FFC0189
:100E600094914A575F4FFA0134913323D1F12223F1
:100E700031F1233021F4809180008F7705C0243038
:100E800031F4809180008F7D8093800018C02130E4
:100E900019F484B58F7704C0223021F484B58F7D96
:100EA00084BD0DC0263021F48091B0008F7705C03D
:100EB000273029F48091B0008F7D8093B000E32F1C
:100EC000F0E0EE0FFF1FEE58FF4FA591B49166239F
:100ED00029F48C91909589238C9308958C91892B7A
:100EE0008C930895682F70E0CB0182559F4FFC01D1
:100EF0002491CB0186569F4FFC0144916A577F4F46
:100F0000FB019491992319F420E030E038C02223AA
:100F100031F1233021F4809180008F7705C0243097
:100F200031F4809180008F7D8093800018C0213043
:100F300019F484B58F7704C0223021F484B58F7DF5
:100F400084BD0DC0263021F48091B0008F7705C09C
:100F5000273029F48091B0008F7D8093B000892FD5
:100F600090E0880F991F84589F4FFC01A591B49180
:100F70008C9120E030E0842311F021E030E0C901C1
:100F800008951F920F920FB60F9211242F933F9343
:100F90004F935F936F937F938F939F93AF93BF9381
:100FA000EF93FF934091C600E091A303F091A40357
:100FB000CF01019660E870E00E94AA0A9C0180912E
:100FC000A5039091A6032817390739F0ED5DFC4F72
:100FD00040833093A4032093A303FF91EF91BF912B
:100FE000AF919F918F917F916F915F914F913F91C1
:100FF0002F910F900FBE0F901F9018955F926F92D8
:101000007F928F929F92AF92BF92CF92DF92EF9298
:10101000FF920F931F93CF93DF93EC013A014B01A3
:10102000413482E458078FE0680780E078070CF0CD
:101030007FC060E874E88EE190E0A40193010E9413
:10104000DF0A2150304040405040CA01B90122E03F
:1010500030E040E050E00E94DF0A59016A01A60139
:101060009501209530954095509594E0220F331FBF
:10107000441F551F9A95D1F760E074E284EF90E029
:101080000E94DF0ACA01B9012FEF30E040E050E0D2
:101090000E948B0AA40193010E94DF0AC9018150BA
:1010A0009F4F181619061CF4522E5A9403C055244B
:1010B0005394521A60E079E08DE390E0A40193012B
:1010C0000E94DF0A2150304040405040CA01B9011F
:1010D00022E030E040E050E00E94DF0A20953095A9
:1010E0004095509583E0220F331F441F551F8A956A
:1010F000D1F760E074E284EF90E00E94DF0ACA0159
:10110000B9012FEF30E040E050E00E948B0AA401CB
:1011100093010E94DF0AC90181509F4F18161906DA
:101120001CF4822F815002C081E0821B851500F5DE
:10113000E885F98581E090E00A8802C0880F991F50
:101140000A94E2F7808360E079E08DE390E0A40107
:1011500093010E94DF0A2150304040405040CA01B4
:10116000B90122E030E040E050E00E94DF0A04C014
:10117000E885F98510829501EC81FD813083EE814F
:10118000FF812083EA85FB85208141E050E0CA0190
:101190000E8402C0880F991F0A94E2F7282B20833F
:1011A000EA85FB852081CA010F8402C0880F991F40
:1011B0000A94E2F7282B2083EA85FB858081088842
:1011C00002C0440F551F0A94E2F7842B8083DF91FD
:1011D000CF911F910F91FF90EF90DF90CF90BF9034
:1011E000AF909F908F907F906F905F900895DC01FB
:1011F0001296ED91FC911397E058FF4F81919191D8
:1012000080589F4F20813181821B930B60E870E0F2
:101210000E94AA0A0895CF93DF93DC011296ED9104
:10122000FC911397EF01CE57DF4F48815981E05869
:10123000FF4F80819181E058F0408417950719F4A1
:101240002FEF3FEF0CC0E40FF51F2081CA0101967C
:1012500060E870E00E94AA0A9983888330E0C9019F
:10126000DF91CF910895FC01A085B18521898C91F2
:1012700090E0022E02C0959587950A94E2F780FFD0
:10128000F6CF0484F585E02D6083089588E891E029
:101290009093A8038093A70383E293E09093AA031B
:1012A0008093A90385EC90E09093AC038093AB030B
:1012B00084EC90E09093AE038093AD0380EC90E0DB
:1012C0009093B0038093AF0381EC90E09093B203CE
:1012D0008093B10386EC90E09093B4038093B303C2
:1012E00084E08093B50383E08093B60387E0809326
:1012F000B70385E08093B80381E08093B903089534
:101300000F931F93CF93DF938C01EB0109C02196BC
:10131000D801ED91FC910190F081E02DC801099573
:1013200068816623A1F7DF91CF911F910F910895F6
:10133000EF92FF920F931F93CF93DF938C017B016A
:10134000EA010CC0D7016D917D01D801ED91FC91AE
:101350000190F081E02DC80109952197209791F720
:10136000DF91CF911F910F91FF90EF9008952F92F1
:101370003F924F925F926F927F928F929F92AF9225
:10138000BF92CF92DF92EF92FF920F931F93DF9362
:10139000CF93CDB7DEB7A0970FB6F894DEBF0FBEE0
:1013A000CDBF1C016A017B01411551056105710525
:1013B00049F4DC01ED91FC910190F081E02D60E3B6
:1013C000099554C0882499245401422E552466243A
:1013D000772401E010E00C0F1D1F080D191DC70137
:1013E000B601A30192010E94BD0AF801608308942E
:1013F000811C911CA11CB11CC701B601A301920163
:101400000E94BD0AC901DA016C017D01C114D10439
:10141000E104F104F1F681E0E82EF12CEC0EFD1E62
:10142000E80CF91C3E010894611C711CD501C40133
:101430000197A109B1096C01C818D90814C0F601B7
:10144000EE0DFF1D60816A3010F4605D01C0695CC3
:10145000D101ED91FC910190F081E02DC101099540
:101460000894E108F1086E147F0449F7A0960FB6BE
:10147000F894DEBF0FBECDBFCF91DF911F910F91CA
:10148000FF90EF90DF90CF90BF90AF909F908F90A4
:101490007F906F905F904F903F902F900895EF92C4
:1014A000FF920F931F93CF93DF93EC017A018B018F
:1014B00077FF0FC0E881F9810190F081E02D6DE2A6
:1014C000099510950095F094E094E11CF11C011D24
:1014D000111DCE01B801A7012AE00E94B709DF91D2
:1014E000CF911F910F91FF90EF900895DC0121158E
:1014F000310541F4ED91FC910190F081E02D642FD4
:10150000099508952A30310519F40E944F0A08956B
:101510000E94B7090895629FD001739FF001829FD6
:10152000E00DF11D649FE00DF11D929FF00D839F72
:10153000F00D749FF00D659FF00D9927729FB00D0F
:10154000E11DF91F639FB00DE11DF91FBD01CF0122
:101550001124089597FB092E07260AD077FD04D0A1
:1015600049D006D000201AF4709561957F4F0895F8
:10157000F6F7909581959F4F0895A1E21A2EAA1B28
:10158000BB1BFD010DC0AA1FBB1FEE1FFF1FA21733
:10159000B307E407F50720F0A21BB30BE40BF50B30
:1015A000661F771F881F991F1A9469F760957095B9
:1015B000809590959B01AC01BD01CF01089597FBEB
:1015C000092E05260ED057FD04D0D7DF0AD0001C07
:1015D00038F450954095309521953F4F4F4F5F4FD0
:1015E0000895F6F790958095709561957F4F8F4F90
:1015F0009F4F0895AA1BBB1B51E107C0AA1FBB1F29
:10160000A617B70710F0A61BB70B881F991F5A958E
:10161000A9F780959095BC01CD010895EE0FFF1FAD
:0C1620000590F491E02D0994F894FFCFA0
:10162C00FF0F010101010101010101010101010192
:10163C00010101010101010101010101010101018E
:10164C00010101010101010101010101010101017E
:10165C00010101010101010101010101010101016E
:10166C0001010101303133340C0D0E0F3235363798
:10167C000B0A090838393A3B070605023F3E3D3C48
:10168C0004030100202123241C1D1E1F22252627B4
:10169C001B1A191828292A2B171615122F2E2D2C28
:0E16AC00141311100000000033098009980982
:00000001FF
